:1018000012C02BC02AC029C028C027C026C025C0AE
:1018100024C023C022C021C020C01FC01EC01DC0C4
:101820001CC01BC01AC011241FBECFE5D4E0DEBF10
:10183000CDBF10E0A0E6B0E0E4E3FEE102C0059019
:101840000D92A036B107D9F711E0A0E6B0E001C0D3
:101850001D92A43AB107E1F7BAC2D2CF0F92AF936B
:10186000BF93CF93DF93EF93FF93FC01EA01DB017A
:10187000C895099231961197D9F7FF91EF91DF91B1
:10188000CF91BF91AF910F9008950F921F920F9338
:10189000AF93BF93CF93DF93EF93FF93FC01EA01E4
:1018A000DB010990199001E043D032961297C9F7F5
:1018B000FC0103E03DD005E03BD0FF91EF91DF91CB
:1018C000CF91BF91AF910F911F900F9008950F93FB
:1018D0001F93EF93FF93FC0103E02AD000E410E094
:1018E000E00FF11FE617F707B9F7FF91EF911F918E
:1018F0000F9108950F930F9222D0082E09E018D06F
:101900000F900F9108950F930F92EF93FF9317D0BD
:10191000FC0160935700C895802DFF91EF910F90C7
:101920000F9108950F930BD001E102D00F9108950C
:10193000E199FECF00935700E895FFFF000000916A
:10194000570000FDFCCF089588E089B98AB188610D
:101950008AB908958AB1877E8AB908958CB95E9B49
:10196000FECF5E9A08958CB1992708958BB199277F
:10197000807890700895EF92FF920F931F93CF930A
:10198000DF937B01C0E0D0E0C617D70760F48C017D
:10199000EDDF8823E9F3E7DFF80181938F012196DA
:1019A000CE15DF05A8F381E090E0DF91CF911F9184
:1019B0000F91FF90EF900895EF92FF920F931F9376
:1019C000CF93DF937C018B01C0E0D0E0C017D1073B
:1019D00030F4F70181917F01C1DF2196F7CF81E0DB
:1019E00090E0DF91CF911F910F91FF90EF900895BC
:1019F00040E050E04817590750F42FEC37E0000062
:101A00002150304037FFFBCF4F5F5F4FF3CF08953A
:101A1000A1DFEEDF0895AADF8823E9F3A4DF803297
:101A200019F481E090E0089585E198DF80E090E08E
:101A3000089590E0282F33272138310589F0223886
:101A4000310524F42038310549F00DC02238310524
:101A500049F02839310539F493E005C092E003C01C
:101A600091E001C092E1892F9927089540E050E06C
:101A70006091A0007091A10046175707D0F4209103
:101A8000A2013091A301E2EAF0E03FBB2EBB2F5F41
:101A90003F4F80818DBBE29AE19AE199FECF4F5F83
:101AA0005F4F31964617570780F33093A301209379
:101AB000A201089540E050E06091A0007091A10063
:101AC00046175707B0F42091A2013091A301E2EA32
:101AD000F0E03FBB2EBB2F5F3F4FE09A8DB3819369
:101AE0004F5F5F4F46175707A0F33093A301209332
:101AF000A2010895CF93DF93C0E0D0E08091A000D1
:101B00009091A100C817D90798F4CE018E559F4F28
:101B10002091A2013091A301220F331FAC0160E498
:101B200070E0C9018C0F9D1FB0DEC05CDF4FE6CFB7
:101B3000F9DEDF91CF9108958091A2019091A301E8
:101B400042EA50E06091A0007091A100880F991FB7
:101B500085DE0895CF93C0E069E081E090E0D3DEB8
:101B6000992784FF02C08F7EC5DE00DF8823E9F35A
:101B7000FADE9927823591051CF5803591050CF028
:101B800054C08134910509F458C0823491057CF425
:101B900081339105B1F18233910524F4C09709F4A2
:101BA00044C010C18034910509F40FC10BC18234C7
:101BB000910509F451C08534910509F450C002C162
:101BC0008635910509F4CDC0873591054CF48235F1
:101BD000910509F44FC08535910509F456C0F2C04E
:101BE0008437910509F48AC0853791052CF4843631
:101BF000910509F461C0E6C08537910509F4A5C0D7
:101C0000E1C009DF882309F4B0CF84E1A7DE81E4D5
:101C1000A5DE86E5A3DE82E5A1DE80E29FDE83E528
:101C20009DDE84E59BDE8BE405C0F5DE882309F4A8
:101C30009CCF84E193DE80E1C6C061E070E080E685
:101C400090E099DEE8DE882309F48FCF84E186DE18
:101C500080916000EEDEEECF64E170E007C061E0ED
:101C600070E080E690E087DE64E070E080E690E07F
:101C700082DEDBCFD0DE882309F477CF60E070E22C
:101C800080E090E024DE4EDED4CF62E070E080E6BB
:101C900090E071DEC0DE882309F467CF20916000F8
:101CA000809161009927982F8827820F911D90932A
:101CB000A3018093A201BDCF63E070E080E690E0D5
:101CC0005ADE20916100809160009927982F882723
:101CD000820F911D9093A1008093A000BC0182EA25
:101CE00090E049DE98DE882309F43FCF80916200BE
:101CF000863411F4FFDE9DCFB9DE9BCF63E070E048
:101D000080E690E038DE20916100809160009927A4
:101D1000982F8827820F911D9093A1008093A00097
:101D20007ADE882309F421CF80916200863411F491
:101D300003DF01C0BFDE84E111DE6091A00070917D
:101D4000A10082EA90E038DE76CF65DE882309F4D0
:101D50000CCF84E103DE8EE101DE83E9FFDD87E065
:101D600069CF64E070E080E690E005DE54DE882311
:101D700009F4FBCE84E1F2DD80916000803531F41E
:101D800080916100882361F4C82F17C0883531F431
:101D900080916100883061F4C3E00FC0803531F478
:101DA00080916100883049F4C2E007C0883529F489
:101DB00080916100882309F4C1E069E08C2F9927A4
:101DC000A2DD38CF85E1CADDD0CECF910895CFE531
:101DD000D4E0DEBFCDBFCEE1F894AEEFB1E021D0CC
:101DE000802D843B61F4AFEFB1E01BD0802D833CAC
:101DF00031F4ADEFB1E015D0802D992781BFA4DD7E
:101E0000B2DD84E690E0F4DDB1DD882311F0A2DEDE
:101E100004C0C150C8BBCC23A1F7FADD80E090E03C
:101E200008C0E199FECFBFBBAEBBE09A11960DB2E0
:041E30000895FFCF43
:0400000300001800E1
:00000001FF
